:10000000F12DFF3FFF3FFF3F063003138312FA003D
:10001000FA0B082800000800031383122230FC00AA
:10002000F801F901FA01FB01FC030319422803104E
:10003000FB0CFA0CF90CF80CF30CF20CF10CF00CB4
:10004000031C1428FC03031934287408F8077508E6
:100050000318750FF90776080318760FFA07770863
:100060000318770FFB0718287408F807750803189A
:10007000750FF90776080318760FFA077708031843
:10008000770FFB0708000313831220088400000881
:10009000F0002108F004200884007008800004208B
:1000A000200884000008F0002208F00520088400E1
:1000B000700880000800031383126D08A3006E0807
:1000C000A400A501A6010130A700080003138312B4
:1000D000FD01F31F7828F009F109F209F309F00A8C
:1000E0000319F10A0319F20A0319F30A8130FD0713
:1000F000F71F8628F409F509F609F709F40A031928
:10010000F50A0319F60A0319F70AFD0A0C207D1CEB
:10011000A028F009F109F209F309F809F909FA0927
:10012000FB09F00A0319F10A0319F20A0319F30A89
:100130000319F80A0319F90A0319FA0A0319FB0A41
:10014000080003138312710DF80DF90D7408F802FD
:100150007508031C750FF902F00DF10D0F30FC004E
:10016000710DF80DF90D7408701CBC28F8027508A3
:10017000031C750FF902C128F80775080318750FDD
:10018000F907F00DF10DFC0BB0287018CD2874089C
:10019000F80775080318750FF907000008007F308D
:1001A000031383126D05F1007108ED00711FED2836
:1001B000200884000008F0002808F00420088400CB
:1001C00070088000200884000008F0002908F0056D
:1001D000200884007008800001292008840000089D
:1001E000F0002A08F005200884007008800020082C
:1001F00084000008F0002B08F00420088400700838
:100200008000080003138312200884000008F00017
:100210002C08F0052D08F0052008840070088000E7
:10022000B8306D04F0002E08840070088000432070
:1002300008007F3003138312ED05200884000008B6
:10024000F0002C08F00520088400700880002008C9
:1002500084000008F0002D08F005200884007008D4
:100260008000BF306D05F0007008ED007017700859
:10027000ED002E088400700880004320080003135E
:100280008312200884000008F0002F08F0042008E2
:10029000840070088000200884000008F000220814
:1002A000F005200884007008800020088400000801
:1002B000F0003008F00420088400700880008030CE
:1002C0002E07F1007108B100710884000008F000E9
:1002D0003208F0047108840070088000200884004F
:1002E0000008F0002108F004200884007008800055
:1002F0002E0884000008ED00200884000008F000AB
:100300002208F0052008840070088000200884007E
:100310000008F0002D08F005200884007008800017
:10032000310884000008F0003308F005310884002B
:10033000700880006D08F000080003138312200885
:1003400084000008F0002208F005200884007008EE
:100350008000200884000008F0002F08F004200826
:10036000840070088000200884000008F0002D0838
:10037000F00520088400700880002E0884006D08B5
:100380008000432008007C34A23492348A347C34C8
:1003900000348434FE34803400348434C234A234D3
:1003A00092348C34423482348A3496346234303419
:1003B00028342434FE3420344E348A348A348A3447
:1003C0007234783494349234923460340234E234A7
:1003D00012340A3406346C349234923492346C34CD
:1003E0000C349234923452343C34003400340034AF
:1003F0000034003440342034103408340434FE34E3
:10040000FE347C3438341034003400340434003486
:100410000034003400340534003400340034003437
:10042000063400340034003400340734003400341F
:10043000FC34223422342234FC34FE34923492349C
:1004400092346C347C348234823482344434FE34CA
:100450008234823444343834FE34923492349234C8
:100460008234FE3412341234123402347C34823436
:1004700082349234F434FE34103410341034FE34A8
:1004800000348234FE348234003440348034823488
:100490007E340234FE341034283444348234FE3442
:1004A0008034803480348034FE340434183404348E
:1004B000FE34FE34083410342034FE347C3482346C
:1004C000823482347C34FE341234123412340C34CC
:1004D0007C348234A2344234BC34FE34123432349C
:1004E00052348C348C3492349234923462340234E8
:1004F0000234FE34023402347E348034803480345A
:100500007E343E344034803440343E347E34803453
:10051000703480347E34C634283410342834C634E1
:100520000E341034E03410340E34C234A234923419
:100530008A3486340800031383122708031DA52A72
:100540000130ED000030EE005B202308F0002408AD
:10055000F1002508F2002608F3006D30F4004E305B
:10056000F500C630F6004130F70066203930F5005E
:100570003030F600F701F8017008F507710803182C
:10058000710FF60772080318720FF7077308031844
:10059000730FF8077708F0007808F100F201F30113
:1005A000FF30F0057F30F1050030F205F3057008EB
:1005B000A3007108A4007208A5007308A600080033
:1005C00003138312FD01F901F80171087004031986
:1005D000003471087506FA00FA1BFD09FB01F51FCE
:1005E000F62AF409F509F40A0319F50AF11FFD2AA0
:1005F000F009F109F00A0319F10A71087504FA000B
:10060000FA1B122BA1207B18252BFD1F0034F009AB
:10061000F109F00A0319F10AF809F909F80A0319AE
:10062000F90A0034F51F212BF11B1D2B7108F9006D
:100630007008F800F101F001052BF101F001F00A5A
:100640000034F109F009FB0A022BF80A0319F90A30
:1006500074087802031D052B75087902031D052B0C
:10066000F901F801F00A0319F10AF11F052B000046
:10067000FF3408007F30031383126705F000700811
:10068000E7003F30E8057008ED00CF206808ED0076
:10069000ED0CED13ED0CED13ED0CED1302216708DD
:1006A000ED0019213F217008EB003F217008EB009D
:1006B0006808ED00ED0CED13ED0CED13ED0CED13F2
:1006C00002216708ED00192107306805F000700865
:1006D000EA007008F1000130F00071080319742B72
:1006E000F00D7010FF3F6E2B7008EA007009EC00EF
:1006F000822B6C08EB058E2B6A08EB048E2B6A08A4
:10070000EB068E2B6908003A0319792B6908013A28
:1007100003197C2B6908023A03197F2B6B08ED0043
:100720009D210800031383125B08AE005408A0004B
:10073000B301FF30B2005508F1000130F00071083C
:100740000319A62BF00D7010FF3FA02B7008A80016
:100750007009AA005608F1000130F0007108031971
:10076000B52BF00D7010FF3FAF2B7008AB00700978
:10077000A9005708F1000130F00071080319C42BDB
:10078000F00D7010FF3FBE2B7008AF007009AC0079
:100790005808F1000130F00071080319D32BF00D57
:1007A0007010FF3FCD2B7008B0007009AD005908E4
:1007B000F1000130F00071080319E22BF00D701008
:1007C000FF3FDC2B7008B4007009B5005A08F10037
:1007D0000130F00071080319F12BF00D7010FF3F8C
:1007E000EB2B7008A1007009A20080305B07F100BC
:1007F0007108B100710884000008F0000030F005B5
:10080000710884007008800080302007F1007108B2
:10081000B100710884000008F0002A08F005710892
:10082000840070088000310884000008F000290866
:10083000F005310884007008800031088400000849
:10084000F0002C08F00531088400700880003108A1
:1008500084000008F0002D08F005310884007008BD
:100860008000310884000008F0003508F0053108E8
:10087000840070088000310884000008F00022081D
:10088000F00531088400700880002008840000080A
:10089000F0003408F004200884007008800020086C
:1008A00084000008F0002C08F0052008840070087F
:1008B0008000200884000008F0002D08F0052008C2
:1008C000840070088000200884000008F0002A08D6
:1008D000F0052008840070088000200884000008CB
:1008E000F0002B08F00420088400700880002E0817
:1008F00084003F30800043202E088400C0308000F8
:100900004320200884000008F0002808F004200894
:10091000840070088000200884000008F000290886
:10092000F00520088400700880002E0884003F3005
:10093000800043202E088400C03080004320053012
:10094000B6000730B700C330B8000130B90030300E
:10095000BA000030BB000800031383122008840093
:100960000008F0002A08F0052B08F0042008840095
:1009700070088000D6015608073C031CCE2C560890
:10098000ED000221D50155083F3C031CCC2C540836
:10099000ED009D21D50AC32CD60ABB2C200884006B
:1009A0000008F0002908F0052808F0042008840059
:1009B00070088000D6015608073C031CEE2C560830
:1009C000ED000221D50155083F3C031CEC2C5408D6
:1009D000ED009D21D50AE32CD60ADB2C08009B22D2
:1009E0000030F4000230F500E02208000313831207
:1009F00056085A02F2005708031C013F5B02F3003D
:100A00007208DD007308DE0054085802DF00550844
:100A1000031C013F5902E00080307306F000803073
:100A20007002031D152D003072020318242D5D087D
:100A3000003CDD005E08031C013FDE01DE02FF30EA
:100A4000E300FF30E400272D0130E300E4018030B3
:100A50006006F00080307002031D302D00305F0210
:100A600003183F2D5F08003CDF006008031C013FB6
:100A7000E001E002FF30E100FF30E200422D0130F2
:100A8000E100E201DD0DDE0D5D10DF0DE00D5F1018
:100A90005408E7005608E8005C08E9003A23803073
:100AA0005E06F000803060067002031D592D5F085D
:100AB0005D020318A62D5F08F0006008F100F10C3C
:100AC000F00CF113711BF11770085D02E50071085D
:100AD000031C013F5E02E60055085906031D722DF6
:100AE000580854060319A52D80306606F0008030A2
:100AF0007002031D7D2D00306502031C8B2D6308E1
:100B0000D60764080318013FD7075F08E502031CF6
:100B1000E6036008E60261085407F0005508031870
:100B2000013F6207F1007008D4007108D5005D082C
:100B3000E5075E080318013FE6077008E70056085E
:100B4000E8005C08E9003A236C2DF02D5D08F00008
:100B50005E08F100F10CF00CF113711BF117700835
:100B60005F02E5007108031C013F6002E6005708C0
:100B70005B06031DBD2D5A0856060319F02D803063
:100B80006606F00080307002031DC82D003065023B
:100B9000031CD62D6108D40762080318013FD5074E
:100BA0005D08E502031CE6035E08E60263085607DB
:100BB000F00057080318013F6407F1007008D600E1
:100BC0007108D7005F08E50760080318013FE607D2
:100BD0005408E7007008E8005C08E9003A23B72DE4
:100BE0000800031383168701903083128700831651
:100BF00086016E30831286000630D400D5010130A4
:100C0000D6000230D7000330D8000530D9000430B8
:100C1000DA000830DB009223D401AC24BC01BD0112
:100C2000BE0180303D06F0008030033A7002031DA3
:100C30001B2EE8303C020318242E9B227008BF00B4
:100C4000BC0A0319BD0A112EBC01BD01BE013E083C
:100C50000A3C031C3A2E3E083F3FD3009B22003043
:100C6000F4000230F500E022530884007008800090
:100C7000BE0A272E80303D06F00080307002031D32
:100C8000432E64303C020318C42EEF247008C900C0
:100C900070083F06031DC32EEF247008CA007008B9
:100CA0004006031DC32EEF247008CB0070084106D8
:100CB000031DC32EEF247008CC0070084206031DEC
:100CC000C32EEF247008CD0070084306031DC32E09
:100CD000EF247008CE0070084406031DC32EEF24D5
:100CE0007008CF0070084506031DC32EEF2470085E
:100CF000D00070084606031DC32EBE0107303E0219
:100D00000318BF2E3C08013FF00000300318013FDC
:100D10003D07F1007008BC007108BD000130700291
:100D2000D4000030031C013F7102D5003E08493F4A
:100D300084000008D6000030D61BFF30D7000030FA
:100D4000D61BFF30D7007008D8007108D9003E08C4
:100D5000013FF000F1010318F10A7008493F8400D7
:100D60000008DA000030DA1BFF30DB000030DA1B4D
:100D7000FF30DB000130DC00F624BE0A7E2E03309B
:100D8000BC070318BD0A3A2E0714C52EFF3FFF3FCC
:02400E007A3FF7
:00000001FF
